:100000000C9434000C9451000C9451000C94510049
:100010000C9451000C9451000C9451000C94E30189
:100020000C9451000C9451000C9451000C94B201AA
:100030000C9451000C9451000C9481010C945100CB
:100040000C9451000C9451000C9451000C945100EC
:100050000C9451000C9451000C9451000C945100DC
:100060000C9451000C94510011241FBECFEFD8E026
:10007000DEBFCDBF11E0A0E0B1E0E2ECF8E002C0ED
:1000800005900D92A834B107D9F711E0A8E4B1E0CA
:1000900001C01D92AD34B107E1F70E944A020C94F1
:1000A0005F040C9400004F925F926F927F928F9248
:1000B0009F92AF92BF92CF92DF92EF92FF920F93F7
:1000C0001F93CF93DF93EC0180917C00857E82604B
:1000D00080937C0080917A00806480937A00809184
:1000E0007A0086FDFCCF609178007091790080E005
:1000F00090E00E94460320E030E040E854E40E9493
:10010000D80320E030EC4FE754E40E94DE026B019C
:100110007C016C837D838E839F8311E028A939A99C
:100120004AA95BA90E94D40387FD10E0812F90E0CB
:100130009FA38EA3111104C0812C912C540106C0E1
:10014000812C912C90E8A92E9FE3B92E8C869D8658
:10015000AE86BF8601E010E02CA93DA94EA95FA99B
:10016000C501B4010E94D40387FF02C000E010E083
:1001700019A308A311E02CA53DA54EA55FA5C701B5
:10018000B6010E94D40387FD10E0812F90E09DA36B
:100190008CA3111104C0412C512C320106C0412CFA
:1001A000512C80E8682E8FE3782E488659866A861F
:1001B0007B8601E010E0A5019401C301B2010E9419
:1001C000D403181614F000E010E01F8F0E8F11E01A
:1001D00028A539A54AA55BA5C701B6010E94D4038D
:1001E00087FD10E0812F90E09BA38AA3111104C02A
:1001F00060E070E0CB0104C060E070E080E89FE365
:10020000688B798B8A8B9B8B01E010E0A3019201B4
:100210000E94D403181614F000E010E01D8F0C8F1C
:10022000FE01EA5BFF4F808191818230910561F090
:100230008330910599F00197C9F416BC80916E0046
:10024000826080936E0016C0109285001092840028
:1002500080916F00826080936F000CC01092B2009A
:100260008091700082608093700004C081E090E013
:100270000E945F0478949FB7F89480914A019FBFD1
:100280008823C9F310924A01EEADFFAD8C8D9D8D90
:10029000892B19F08081826002C080818D7F8083EC
:1002A000FE01E05CFF4F0190F081E02D8E8D9F8D6F
:1002B000892B19F08081846002C080818B7F8083CC
:1002C000FE01EE5BFF4F0190F081E02D88A199A126
:1002D000892B19F08081886002C08081877F8083AC
:1002E000DF91CF911F910F91FF90EF90DF90CF9012
:1002F000BF90AF909F908F907F906F905F904F9046
:1003000008951F920F920FB60F9211242F933F93CF
:100310008F939F938091480190914901019690930A
:1003200049018093480180914A01813091F02091E8
:1003300048013091490180914B0190914C0128175F
:10034000390738F081E080934A01109249011092F8
:1003500048019F918F913F912F910F900FBE0F9069
:100360001F9018951F920F920FB60F9211242F9382
:100370003F938F939F9380914801909149010196FB
:10038000909349018093480180914A01813091F016
:10039000209148013091490180914B0190914C018D
:1003A0002817390738F081E080934A0110924901FB
:1003B000109248019F918F913F912F910F900FBE06
:1003C0000F901F9018951F920F920FB60F92112445
:1003D0002F933F938F939F93809148019091490170
:1003E0000196909349018093480180914A018130A0
:1003F00091F0209148013091490180914B019091F9
:100400004C012817390738F081E080934A01109297
:100410004901109248019F918F913F912F910F9028
:100420000FBE0F901F901895ECE7F0E02081206C34
:100430002083EAE7F0E0208127682083FC0115AEE5
:1004400014AE239AEE5BFF4F25E230E03183208328
:10045000229A329731832083219AFC0137AF26AF4D
:1004600025B5236025BDEC5BFF4F41E050E0518393
:1004700040832AE030E030934C0120934B0124B5B7
:10048000226024BD29EF27BD32965183408380E04E
:1004900090E00895CF92DF92EF92FF9280E091E09A
:1004A0000E941402C12CD12C760160E070E0CB01D7
:1004B0006093000170930101809302019093030106
:1004C00080E091E00E9453008FEFC81AD80AE80A32
:1004D000F80AC701B6010E9446032FE632E143E065
:1004E0005BE30E94D80320E030E0A9010E947A0279
:1004F000DFCF5058BB27AA270ED01CC10DD130F03A
:1005000012D120F031F49F3F11F41EF402C10EF419
:10051000E095E7FBF8C0E92F1ED180F3BA17620718
:1005200073078407950718F071F49EF536C10EF431
:10053000E0950B2EBA2FA02D0B01B90190010C01F3
:10054000CA01A0011124FF27591B99F0593F50F40B
:10055000503E68F11A16F040A22F232F342F442763
:10056000585FF3CF469537952795A795F04053955B
:10057000C9F77EF41F16BA0B620B730B840BBAF02B
:100580009150A1F0FF0FBB1F661F771F881FC2F796
:100590000EC0BA0F621F731F841F48F487957795AA
:1005A0006795B795F7959E3F08F0B3CF9395880F61
:1005B00008F09927EE0F9795879508950CD0BAC04B
:1005C000B2D040F0A9D030F021F45F3F19F09BC0C9
:1005D0005111E4C09EC0BFD098F39923C9F35523AD
:1005E000B1F3951B550BBB27AA2762177307840726
:1005F00038F09F5F5F4F220F331F441FAA1FA9F3DC
:1006000033D00E2E3AF0E0E830D091505040E695CD
:10061000001CCAF729D0FE2F27D0660F771F881F2E
:10062000BB1F261737074807AB07B0E809F0BB0B1D
:10063000802DBF01FF2793585F4F2AF09E3F510541
:1006400068F061C0ABC05F3FECF3983EDCF3869589
:1006500077956795B795F7959F5FC9F7880F911DB7
:100660009695879597F90895E1E0660F771F881FA3
:10067000BB1F621773078407BA0720F0621B730B56
:10068000840BBA0BEE1F88F7E0950895E89409C033
:1006900097FB3EF490958095709561957F4F8F4FB5
:1006A0009F4F9923A9F0F92F96E9BB279395F695CB
:1006B000879577956795B795F111F8CFFAF4BB0F49
:1006C00011F460FF1BC06F5F7F4F8F4F9F4F16C0AD
:1006D000882311F096E911C0772321F09EE8872F37
:1006E000762F05C0662371F096E8862F70E060E0F3
:1006F0002AF09A95660F771F881FDAF7880F96956C
:10070000879597F9089597F99F6780E870E060E012
:1007100008959FEF80EC089500240A94161617069A
:1007200018060906089500240A94121613061406E2
:1007300005060895092E0394000C11F4882352F045
:10074000BB0F40F4BF2B11F460FF04C06F5F7F4FFD
:100750008F4F9F4F089557FD9058440F551F59F0E4
:100760005F3F71F04795880F97FB991F61F09F3F9E
:1007700079F087950895121613061406551FF2CFC7
:100780004695F1DF08C0161617061806991FF1CF17
:1007900086957105610508940895E894BB2766273E
:1007A0007727CB0197F9089566D008F48FEF089565
:1007B0000BD0C0CFB1DF28F0B6DF18F0952309F0D9
:1007C000A2CFA7CF1124EACFC6DFA0F3959FD1F324
:1007D000950F50E0551F629FF001729FBB27F00DEF
:1007E000B11D639FAA27F00DB11DAA1F649F662744
:1007F000B00DA11D661F829F2227B00DA11D621F93
:10080000739FB00DA11D621F839FA00D611D221F4C
:10081000749F3327A00D611D231F849F600D211D30
:10082000822F762F6A2F11249F5750408AF0E1F0D3
:1008300088234AF0EE0FFF1FBB1F661F771F881F1C
:1008400091505040A9F79E3F510570F05CCFA6CF64
:100850005F3FECF3983EDCF3869577956795B79507
:10086000F795E7959F5FC1F7FE2B880F911D969531
:10087000879597F90895990F0008550FAA0BE0E89E
:10088000FEEF16161706E807F907C0F01216130652
:10089000E407F50798F0621B730B840B950B39F492
:1008A0000A2661F0232B242B252B21F408950A26F8
:1008B00009F4A140A6958FEF811D811D0895F8943C
:0208C000FFCF68
:1008C2000000000000000000000000000000000026
:1008D2000000000000000000000000000000000016
:1008E2000000000000000000000000000000A04323
:1008F200000061440000003F0AD7233C00000000D2
:080902000000000000000000ED
:00000001FF
